:020000040000FA
:040000000230722830
:08000800A0000308A100AE08EE
:100010000319AD03AE0B1928AD08031D19280F30C5
:10002000AD004230AE004030AF070318AE0A0130D9
:10003000AC000B11831221088300A00E200E0900D2
:10004000A20A0A302202031C52280030A200A30A8E
:1000500006302302031C52280030A200A300A40A89
:100060000A302402031C52280030A400A50A0630DE
:100070002502031C52280030A400A500A60A270E62
:100080002604AA0013302A0203184E280A3026023A
:10009000031C52280030A600A70A52280130A600EF
:1000A0000030A700230E22048600051402306E20C3
:1000B0000510250E24048600851402306E2085105C
:1000C000270E26048600051502306E200511FF302C
:1000D0008600003085000030AC000800AB00AB0BA0
:1000E0006F2808000030AC000830A2000530A300E3
:1000F0000930A4000530A5000230A6000130A70099
:100100000F30AD004330AE004030AF000030AA00E9
:100110000030AB00031383160030860018308500D2
:10012000C03081008312810100308500FF308600DD
:10013000A0308B002C182020050829061839031937
:100140009A28A906A0306E200508A900A91DC0287C
:10015000291EAB289A28A60A270E2604AA001330C7
:100160002A020318BB280A302602031CD0280030BC
:10017000A600A70AD0280130A6000030A700D0288A
:10018000A40A0A302402031CD0280030A400A50AC7
:1001900006302502031CD0280030A400A500D0287A
:0401A00052209A2827
:02400E00F13F80
:00000001FF
